:020000040800F2
:1000000030410020A101000863190008D71700083B
:1000100061190008910800089D1E000800000000FA
:100020000000000000000000000000006719000848
:10003000930800080000000065190008691900080D
:10004000BB010008BB010008BB010008BB010008A0
:10005000BB010008BB010008BB010008BB01000890
:10006000BB010008BB010008BB010008BB01000880
:10007000BB010008BB010008BB010008BB01000870
:10008000BB010008BB010008BB010008BB01000860
:10009000BB010008BB010008BB010008BB01000850
:1000A000BB010008BB010008BB010008BB01000840
:1000B000BB010008BB010008BB010008BB01000830
:1000C000BB010008BB010008BB010008BB01000820
:1000D000BB010008851E0008911E0008BB01000836
:1000E000BB010008BB010008BB010008BB01000800
:1000F000BB010008BB010008BB010008BB010008F0
:10010000BB010008BB010008BB010008BB010008DF
:10011000411A0008BB010008BB010008BB01000830
:10012000BB010008BB010008BB010008BB010008BF
:10013000BB010008BB010008BB010008BB010008AF
:10014000BB010008BB010008BB010008BB0100089F
:10015000BB010008BB010008BB010008BB0100088F
:10016000BB010008BB010008BB010008BB0100087F
:10017000BB010008BB010008BB0100080000000033
:10018000BB010008BB010008DFF810D000F0DAFA6C
:1001900000480047DD1E0008AFF30080304100201A
:1001A0000648804706480047FEE7FEE7FEE7FEE711
:1001B000FEE7FEE7FEE7FEE7FEE7FEE7ED190008D3
:1001C000890100082DE9F05F0546002092469B4614
:1001D00088460646814640241BE02846414647465D
:1001E000224600F0F8F953465A46C01A914110D3FE
:1001F00011461846224600F0DFF92D1A67EB010878
:100200004F4622460120002100F0D6F917EB0009E5
:100210004E41201EA4F10104DFDC484631462A4647
:100220004346BDE8F09FD2B201E000F8012B491E21
:10023000FBD270470022F6E710B513460A46044683
:100240001946FFF7F0FF204610BD2DE9FE4F80460E
:1002500081EA0300C00F0C46009021F0004123F01A
:100260000045B8EB0200A94105D240462146904620
:100270001C460B46024623F00040104347D0270D92
:10028000C7F30A00C3F30A510290401A01904028B4
:100290006BDAC3F3130040F4801B0098924620B140
:1002A0000023D2EB030A63EB0B0B01985946C0F114
:1002B0004002504600F080F906460D465046594629
:1002C000019A00F098F910EB08006141002487EAD8
:1002D000115284EAE7731A4340D0009A62B3019A3C
:1002E000012A4FEA075215DC001B61EB02014FF0B7
:1002F000004202EA0752CDE90042001C41F580119C
:1003000032462B4600F0CFF903B0BDE8F08F4046EF
:100310002146F9E7001B61EB0201001C41F5801347
:1003200000185B412018A2F5001747EB030140EAD3
:10033000D570B6196D4111E06D084FEA360645EAF1
:10034000C0754FEA0752001B61EB0201001C41F52A
:10035000801149084FEA30000019514132462B46BE
:1003600003B0BDE8F04F00F08FB9009801224000C3
:100370000023D0EB020263EBE073009821464FEAC2
:10038000E074B8EB000061EB0401E9E783F000439F
:100390005BE781F0004158E72DE9FE4F81EA030455
:1003A00004F0004421F0004100944FF0000B23F0D2
:1003B000004350EA01045ED052EA03045BD0C3F369
:1003C0000A54C1F30A552C44A4F2F3340194A0FB5F
:1003D0000254C1F3130141F48011C3F3130343F436
:1003E000801301FB024400FB034E840A970A44EA8F
:1003F000815447EA8357A4FB076802958D0A05FBE1
:1004000007854FEA932C04FB0C542705029D4FEA05
:10041000065847EA1637B5EB08056EEB070C870E52
:10042000920E47EA811742EA8312A7FB0201B6EB5C
:100430000B0164EB00042B0D43EA0C335E1844EB14
:100440001C50DA465146E7FB0201C5F313044FEA9C
:100450000B3343EA14534FEA0432019C43EA060388
:10046000A4F10C040294009CCDE900B400F01BF947
:1004700003B0BDE8F08F00200146F9E72DE9F04D0B
:1004800081EA030404F0004B21F0004514464FF0CC
:10049000000A23F0004150EA050220D054EA01028C
:1004A0001DD0C5F30A570246C5F31303C1F3130069
:1004B000C1F30A5640F4801543F48013A7EB0608F5
:1004C000101BD64608F2FD3873EB050002D308F185
:1004D000010801E092185B41B8F1000F03DA002037
:1004E0000146BDE8F08D00204FF480110646844699
:1004F0000EE0171B73EB050705D3121B63EB050317
:1005000006434CEA010C49084FEA300092185B415F
:1005100050EA0107EDD152EA030012D082EA04004A
:1005200083EA0501084305D0101BAB4106D2012226
:10053000002306E000224FF0004302E06FF00102CA
:1005400053101AEB06004CEB085110EB0A0041EB7C
:100550000B01BDE8F04D00F097B800F0004230F01C
:1005600000400AD0C10D01F56071C0F3160042EAE7
:100570000151C208400711437047002001467047EF
:1005800001F0004330B421F0004150EA010206D0EE
:100590000A0DA2F56072C1F31301002A02DC30BC1F
:1005A00000207047440F44EAC104C100E01830BC89
:1005B00000EBC25000F031B8202A04DB203A00FAE8
:1005C00002F1002070479140C2F1200320FA03F3AA
:1005D000194390407047202A04DB203A21FA02F0A8
:1005E0000021704721FA02F3D040C2F1200291406D
:1005F000084319467047202A06DBCB17203A41FAF8
:1006000002F043EAE07306E041FA02F3D040C2F19F
:10061000200291400843194670470029A8BF70473F
:10062000401C490008BF20F00100704710B4B0FA28
:1006300080FC00FA0CF050EA010404BF10BC7047C3
:1006400049B1CCF1200421FA04F411FA0CF118BFDD
:10065000012121430843A3EB0C01CB1D4FEA0061AC
:100660004FEA102042BF002010BC704700EBC3507F
:1006700010440029A4BF10BC7047401C490008BFAB
:1006800020F0010010BC704710B5141E73F1000477
:1006900008DA401C41F1000192185B411A4301D174
:1006A00020F0010010BD2DE9F04D92469B4611B19E
:1006B000B1FA81F202E0B0FA80F220329046FFF700
:1006C0007BFF04460F4640EA0A0041EA0B0153460D
:1006D0005A46084313D0114653EA010019D0C8F115
:1006E00040025046FFF777FF05460E4650465946F2
:1006F0004246FFF761FF084305D0012004E0204691
:100700003946BDE8F08D0020054346EAE0762C43EB
:1007100037430A986305E40AA0EB08000022FD0AAB
:1007200044EA47540A3002D500200146E9E70105B2
:1007300010196941DDE9084500196941BDE8F04D2E
:10074000A2E70000064C074D06E0E06840F0010318
:1007500094E8070098471034AC42F6D3FFF718FD31
:100760000020000820200008464910B54A6822F4FD
:1007700040324A604A6843681A434A6001684A68DE
:1007800022F480724A6001684A68036942EA0322DF
:100790004A6001684A6822F040724A6001684A680B
:1007A00083681A434A6001688A6822F400628A609A
:1007B00001688A68C3681A438A60816A6FF0706250
:1007C000D14201688A6822F070628A6001688A6892
:1007D0000CD0836A1A438A6001688A6822F040520A
:1007E0008A6001688A68C36A1A4301E022F04052B5
:1007F0008A6001688A6822F002028A6001688A6859
:10080000037E42EA43028A6090F8201000290168C2
:100810004A680FD042F400624A6001684A6822F4D4
:1008200060424A6001684A68174C436A04EB4333EC
:100830001A4301E022F400624A600168CA6A22F4A5
:100840007002CA620168CA6A838B104C04EB0353BE
:100850001A43CA6201688A6822F400728A600168D9
:100860008A6890F8303042EA43228A6001688A68D8
:1008700022F480628A6001688A68406942EA8020C6
:10088000886010BD0023014000E0FFFF0000F0FF82
:10089000FEE770477047000078B50024009490F898
:1008A0003C20012A19D0012280F83C200A68072345
:1008B0000568092A13D9EE680A3A02EB420293400E
:1008C0009E43EE600B788A680A3B03EB43039A4031
:1008D0000368DD682A43DA6010E0022078BD2E69E3
:1008E00002EB420293409E432E610B788A6803EB31
:1008F00043039A4003681D692A431A614A681F230B
:10090000072A13D205686E6B521E02EB82029340D7
:100910009E436E630B790A885B1E92B203EB8303DE
:100920009A4003685D6B2A435A6327E005680D2AE5
:1009300012D22E6BD21F02EB820293409E432E6393
:100940000B790A88DB1F92B203EB83039A4003689A
:100950001D6B2A431A6311E0EE6A0D3A02EB820224
:1009600093409E43EE620B790A880D3B92B203EBF3
:1009700083039A400368DD6A2A43DA62164B0568EE
:10098000144A9D4206D10D68122D03D1556845F4D5
:100990008005556005689D4218D10B68102B01D069
:1009A000112B13D1536843F40003536009681029D5
:1009B0000CD10A490A4A0968B1FBF2F101EB810145
:1009C000490000E0491E00910029FBD180F83C401D
:1009D000002078BD002301400020014024000020B9
:1009E00040420F00006C70470068C06C704770B5E3
:1009F00004004FF0000503D0206C002610B107E082
:100A0000012070BD204600F01DF8666484F83C604B
:100A1000206CC00610D4206C20F4885040F00200F6
:100A200020642046FFF7A0FE6664206C20F00200E0
:100A300040F00100206400E0012584F83C60284675
:100A400070BD000010B586B0044614216846FFF75B
:100A5000F1FB1149206888421CD11048002102682E
:100A600042F480720260006800F4807005900B48C8
:100A70001438026842F001020260006800F00100D0
:100A80000590102000900320CDE90101694604483B
:100A900000F0F4F806B010BD0020014044380240D8
:100AA000000002402DE9F041044600680D468168CF
:100AB0004FF0000749050BD58068C00508D5206CAC
:100AC00040F02000206484F83C700120BDE8F081F3
:100AD00000F0B2F906460FE0681C0DD025B100F019
:100AE000ABF9801BA84207D9206C40F004002064B9
:100AF00084F83C700320E9E7206800688007EBD5A4
:100B000021686FF012000860206C40F400702064CF
:100B10002068816811F0405F13D1217E89B9C16AD4
:100B200011F4700F02D0806840050AD4206C20F4C4
:100B300080702064206CC00403D4206C40F001005D
:100B400020640020C2E7000018B50021009190F851
:100B50003C20012A07D0012280F83C2002689368DB
:100B6000DB0702D011E0022018BD936843F00103B7
:100B700093602A4A2A4B1268B2FBF3F202EB42025C
:100B800000E0521E0092002AFBD102689368DB0746
:100B900041D0036C40F20164A34343F480730364C7
:100BA00053685B0505D5036C23F4005343F480536D
:100BB0000364036CDB0404D5436C23F00603436435
:100BC00000E0416480F83C1016496FF02203136086
:100BD00049680068CA06144906D088421BD181685A
:100BE00011F0405F13D016E08842F8D00F4A9042CF
:100BF00003D1D1F80423D206F1D00D4A90420AD194
:100C0000D1F8041301F01F011029E8D303E0816833
:100C100041F080418160002018BD000024000020C8
:100C200040420F000023014000200140002101400C
:100C30000022014090F83510022903D0802141653F
:100C400001207047052180F835100068016821F007
:100C5000010101600020704770B5044600F0ECF817
:100C60000546601C02D004480078044400F0E4F813
:100C7000401BA042FAD370BD180000202DE9F84FA8
:100C8000DFF87CB100224FF001084FF0030A4FF06B
:100C90000F090BF1040E00BF0B6808FA02F42340A1
:100CA000A3426ED14D68022D01D0122D0ED1D50870
:100CB00000EB850CDCF820505607F70E09FA07F612
:100CC000B5430E69BE402E43CCF82060066855003F
:100CD0000F790AFA05FC07F0030726EA0C06AF4075
:100CE000374307604E68012E05D0022E03D0112E27
:100CF00001D0122E0ED18668CF6826EA0C06AF40CE
:100D0000374387604668A6430C79C4F300149440C7
:100D100034434460C6688C6826EA0C06AC40344311
:100D2000C4604C68E40065D5364C256845F48045C0
:100D30002560246822F0030504F480440094324CBA
:100D40002E19D6F8084895072F0F09FA07F5AC4376
:100D50002E4DA84201D1002524E02D4DA84201D1FD
:100D600001251FE02B4DA84201D102251AE02A4D92
:100D7000A84201D1032515E0284DA84202D104253F
:100D800010E037E0264DA84201D105250AE0254DA7
:100D9000A84201D1062505E0234DA84201D107252F
:100DA00000E00825BD402543C6F80858DBF80040A0
:100DB0005D464E689C43F60300D51C432C60DEF86C
:100DC000004075464E689C43B60300D51C432C601A
:100DD0000B4D08352C684E689C43F60200D51C4329
:100DE0002C60074D0C352C684E689C43B60200D52C
:100DF0001C432C60521C102AFFF44EAFBDE8F88F44
:100E0000003C0140443802400030014000000240F4
:100E10000004024000080240000C024000100240A2
:100E20000014024000180240001C02400AB1816117
:100E300070470904FBE70000014880687047000024
:100E400018000020024881680278114481607047D0
:100E5000180000200B4810B5016841F400710160D2
:100E6000016841F480610160016841F480710160B2
:100E7000032000F06FF8002000F006F800F024F8DE
:100E8000002010BD003C024070B50D4D04464FF4EB
:100E90007A712878B1FBF0F00A490968B1FBF0F0EB
:100EA00000F0E2FA48B9102C07D200222146501E69
:100EB00000F030F800206C6070BD012070BD0000B3
:100EC00018000020240000200A4808B5016841F4F9
:100ED00080410160006800F4804000900548001FD8
:100EE000016841F080510160006800F0805000907E
:100EF00008BD000044380240002809DB00F01F0252
:100F0000012191404009800000F1E020C0F800116B
:100F100070470000F0B40E4B1B680C46C3F302236D
:100F2000C3F10705042D00D90425191D072901D295
:100F3000002300E0DB1E012606FA05F1491E2140D0
:100F400099409E40761E16403143F0BC00F0A7BF8A
:100F50000CED00E0064900F0070208684FF6FF03B9
:100F6000184040EA0220034A10430860704700001E
:100F70000CED00E00000FA052DE9F0470E460500F3
:100F800065D0DFF81481D8F80000F7B200F00F0048
:100F9000B04207D288F80070D8F8000000F00F00C7
:100FA000B04254D128683D4C810712D5400703D583
:100FB000206840F4E05020602878000703D52068BE
:100FC00040F4604020602068A96820F0F0000843E9
:100FD00020602878C0072DD030496868083901287A
:100FE00012D0022813D0032811D0096889070029DC
:100FF0002DDA216821F0030101432160FFF71CFF76
:10100000814641F2883A0EE009688903EFE70968F2
:101010008901ECE7FFF710FFA0EB0901514502D968
:101020000320BDE8F0872068696800F00C00B0EB91
:10103000810FEFD1D8F80010404601F00F01B14206
:1010400007D90770006800F00F00B04201D00120FE
:10105000E7E72878400705D52068E96820F4E050E4
:10106000084320602878000706D52068296920F405
:10107000604040EAC100206000F036F82168084A6C
:10108000C1F30311515CC840064908600020FFF716
:10109000FBFE0020C5E70000003C0240083802408B
:1010A000E81F00082400002004480549006809687A
:1010B000044AC1F38221515CC840704724000020DB
:1010C00008380240F81F000804480549006809680C
:1010D000044AC1F34231515CC840704724000020EB
:1010E00008380240F81F0008154810B5006810F0D5
:1010F0000C02144813D01449042A0FD0082A0ED128
:101100000F4C241F2268236802F03F025B0207D5C0
:101110002068C0F38810A0FB010106E0084610BD5E
:101120002168C1F38811A1FB00010023FFF74AF8F1
:101130002168C1F30141491C4900B0FBF1F010BD29
:10114000083802400024F40040787D012DE9F84F72
:10115000050076D02878DFF8F8B2BE4CC00749D039
:10116000DBF800105846C1F38101012908D000685E
:10117000C0F3810002280AD1201D0068400206D574
:101180002068800336D568680028E2D032E06868BD
:10119000B0F5803F10D0B0F5A02F206810D020F41B
:1011A00080302060206820F4802020606868A0B132
:1011B000FFF742FE06460CE0206840F48030F4E77A
:1011C00040F480202060F7E7FFF736FE801B64289C
:1011D00073D820688003F7D50CE0FFF72DFE064694
:1011E00005E000BFFFF728FE801B6428F0D82068C8
:1011F0008003F7D42878DFF8608280074FF0000979
:101200003ED5DBF80010584611F00C0F09D00068ED
:10121000C0F3810002280BD18D48001F00684002F6
:1012200006D42068800715D5E868012809D111E0A7
:10123000E868B8B10120C8F80000FFF7FDFD0646D8
:1012400005E002E1FFF7F8FD801B0228C0D8206806
:101250008007F7D52068296920F0F80040EAC1002E
:1012600020600DE0C8F80090FFF7E6FD064604E0B8
:10127000FFF7E2FD801B02281FD820688007F7D403
:101280002878000722D5724E744869696C3671B1AE
:1012900001210160FFF7D0FD074604E0FFF7CCFD18
:1012A000C01B022809D830688007F7D50EE0C0F8C7
:1012B0000090FFF7C1FD074605E083E0FFF7BCFDA6
:1012C000C01B02287ED830688007F7D428784007F2
:1012D00068D5DFF87CA100270AF1380ADAF80000A7
:1012E000C0000BD4DAF8001041F08051CAF80010A9
:1012F000DAF80000012700F080500090584E306866
:10130000C00510D4306840F480703060FFF794FD61
:10131000009005E0FFF790FD0099401A022851D88F
:101320003068C005F6D54A4EA868683601280FD047
:101330000528306810D020F001003060306820F0BF
:1013400004003060A868B8B1FFF776FD00900FE0A8
:10135000306840F00100F4E740F004003060F7E747
:10136000FFF76AFD0099411A41F28830814264D842
:1013700030688007F4D50EE0FFF75EFD009007E0CF
:10138000FFF75AFD0099411A41F28830814254D842
:1013900030688007F4D42FB1DAF8001021F08051C2
:1013A000CAF80010A869C0B3DBF80010C1F38101CE
:1013B00002294AD00228484607D0C8F86000FFF743
:1013C0003BFD00E039E005463AE04746C8F86000DA
:1013D000FFF732FD064604E0FFF72EFD801B0228D2
:1013E0002BD820688001F7D4D5E907010843A96A02
:1013F0001C4A490802EB01416A6A41EA821108432A
:1014000095F82C1040EA01611148001F016001208D
:101410003866FFF711FD054605E014E0FFF70CFD07
:10142000401B022809D820688001F7D50BE000BFD7
:10143000FFF702FD401B022802D90320BDE8F88F08
:1014400020688001F4D40020F8E70120F6E70000CE
:10145000083802400038024000004742800E4742F0
:10146000007000400000FFFF10B5401EB0F1807F0B
:1014700001D3012010BD4FF0E02460610F216017FF
:1014800000F00DFD0020A06107202061002010BDAC
:101490007047000070B5026804461068D16853694F
:1014A00010F00F0F50D003F0010501F49076354392
:1014B0005DD0C20705D0CA0503D5E26B42F0010238
:1014C000E263420705D5DA0703D0E26B42F002027D
:1014D000E263820705D5DA0703D0E26B42F004022B
:1014E000E263020705D5DA0703D0E26B42F0080297
:1014F000E263E26B002A33D0800604D5880602D569
:10150000204600F0B9FA20684069E16BC0F3801012
:10151000090700D428B3204600F0A0FA20684169EA
:1015200049061AD5416921F040014161606BA0B1C3
:101530001B490165606BFFF77DFB002810D0606BD5
:10154000016DBDE870400847830610D58B060ED5A7
:101550002046BDE8704000F08FBA2046FFF798FFA4
:1015600070BD2046FFF794FF0020E06370BD0306C6
:1015700006D50B0604D52046BDE8704000F01EBC21
:101580004006F3D54806F1D5D168204621F0400148
:10159000D160202184F8391000F01CF970BD0000E2
:1015A0004D1A000870B5040004D094F839000025E5
:1015B00010B106E0012070BD84F83850204600F0DC
:1015C00023F8242084F839002068C16821F40051F0
:1015D000C160204600F09CFA2068016921F4904126
:1015E00001612068416921F02A0141612068C168D8
:1015F00041F40051C160E563202084F8390084F88B
:101600003A00002070BD0000F0B587B004461421F8
:101610006846FEF70FFE3A48384E256838491038BC
:10162000022201230324B5421FD10D6845F4002591
:101630000D60096801F400210591016841F0040181
:1016400001600068694600F004000590A0028DE882
:101650001D00082004902B48FFF710FB00221146C4
:101660003420FFF757FC342022E0274F0726BD42E5
:1016700022D12349091D0D6845F010050D60096848
:1016800001F010010591016841F00201016000685C
:10169000694600F002000590C0208DE85D001B48FF
:1016A000FFF7ECFA002211462520FFF733FC252036
:1016B000FFF722FC07B0F0BD154FBD42FAD10D680F
:1016C00045F400350D60096801F4003105910168A9
:1016D00041F0080101600068694600F008000590CB
:1016E00060208DE85D000B48FFF7C8FA0022114624
:1016F0002620FFF70FFC2620DAE70000004C004010
:10170000403802400008024000100140000402403E
:1017100000440040000C024070472DE9F8430446A5
:1017200090F839001F4616460D46202850D1A5B125
:101730009EB194F8380001284AD0012084F838007E
:101740004FF00008C4F83C80212084F83900FFF7EE
:1017500073FBA6848146E68426E00120BDE8F88379
:10176000E08C401EE084A0684B46B0F5805F4FF0EF
:1017700000024FF080012046009703D000F04FFB9D
:10178000E8B90DE000F04BFBC8B928882168C0F328
:1017900008004860206908B16D1C05E0AD1C03E03D
:1017A000216815F8010B4860E08C0028D8D14B4621
:1017B000002240212046009700F031FB08B10320B1
:1017C000CCE7202084F8390084F838800020C5E771
:1017D0000220C3E77047FEE77FB500241448009459
:1017E0000194029411490394C0E9001484600461D7
:1017F000047680F820400F49C0E90A140125C5612C
:10180000C46080F830404561FFF7F1F808B1FFF798
:1018100041F80420CDE90005694602940448FFF729
:101820003BF8002801D0FFF735F87FBD00200140CC
:10183000280000200100000F70B586B01421684612
:10184000FEF7F8FC1A480024016841F0010101602C
:10185000016801F001010591016841F00801016092
:10186000016801F008010591016841F0040101607F
:10187000016801F004010591016841F00201016075
:1018800000680C4E00F002004FF4704505900022F5
:1018900029463046FFF7CAFA01200095CDE9010438
:1018A000694630460394FFF7E9F906B070BD0000C1
:1018B00030380240000C02400C4810B50A49016063
:1018C0004FF4E1314160002181600C22C160C0E928
:1018D00004128161C161FFF765FE002803D0BDE8F5
:1018E0001040FEF7D7BF10BD004C00407000002034
:1018F0000C4810B50A4901604FF4E1314160002104
:1019000081600C22C160C0E904128161C161FFF7EE
:1019100049FE002803D0BDE81040FEF7BBBF10BD54
:1019200000100140B00000200C4810B50A490160C9
:101930004FF416414160002181600C22C160C0E972
:1019400004128161C161FFF72DFE002803D0BDE8BC
:101950001040FEF79FBF10BD00440040F000002083
:10196000FEE7704770477047FFF76CBA30B593B029
:1019700030216846FEF75EFC14210CA8FEF75AFCE5
:1019800018480025016841F080510160006800F0AE
:10199000805011901448016841F480410160006852
:1019A000022400F480401190012003901020049044
:1019B000009406940820CDE907504820CDE9090499
:1019C00003200B906846FFF7C1FB0CA90F2081E8AC
:1019D0003100E002CDE90F0502210CA8FFF7CCFA97
:1019E00013B030BD4038024000700040104801681C
:1019F00041F4700101600F48016841F0010101608C
:101A00000C4A00210832116002680B4B1A40026038
:101A1000031D0A4A1A60026822F480220260054807
:101A20000C30016002495806803908607047000098
:101A300088ED00E000380240FFFFF6FE1030002481
:101A40000148FFF727BD00007000002010B5806B33
:101A50000021C185C184FFF71BFD10BD0168CA6864
:101A600022F49072CA6001684A6922F001024A6158
:101A7000202180F83A10704710B590F83A102229CA
:101A800001D0022010BD8168B1F5805F11D00169DD
:101A9000002901681FD0496801F07F03816A4A1C50
:101AA00082620B70C18D491E0904090CC18518D0D2
:101AB0002BE00269816A002A0268526805D0D2B21E
:101AC0000A80816A491C8162ECE7C2F308020A803D
:101AD000816A891CF7E74A68816A4B1C83620A7035
:101AE000E0E70168CA6822F02002CA600168CA689B
:101AF00022F48072CA6001684A6922F001024A61D8
:101B0000202180F83A10FFF707FE002010BD0000EA
:101B10002DE9F041044600680169E26821F4405172
:101B2000114301612169A068E269084361691143B9
:101B300022680843D16849F20C6399430143D1609C
:101B400020684169A26921F4407111434161E26951
:101B50006425B2F5004F9748974922684FF0320844
:101B60003FD08A4201D082427CD1FFF7ADFA00EB30
:101B7000C00101EB001061688900B0FBF1F6FFF7CE
:101B8000A3FA00EBC00101EB001061688900B0FB13
:101B9000F1F0B0FBF5F06FF01801484306EB80015F
:101BA00008EB0110B0FBF5F000F0F006FFF78CFA3F
:101BB00000EBC00101EB001061688900B0FBF1F09F
:101BC000B0FBF5F006EB0016FFF77EFA00EBC00164
:101BD00001EB001061688900B0FBF1F7FFF774FAC0
:101BE000D2E08A4201D082423DD1FFF76DFA00EB8C
:101BF000C00101EB001061684900B0FBF1F0B0FBDF
:101C0000F5F00601FFF760FA00EBC00101EB0010F0
:101C100061684900B0FBF1F7FFF756FA00EBC0012D
:101C200001EB001061684900B0FBF1F0B0FBF5F08A
:101C30006FF01801484307EB800108EBC100B0FBCF
:101C4000F5F000F0F80006EB4006FFF73DFA00EB78
:101C5000C00101EB001061684900B0FBF1F7FFF72C
:101C600033FA3CE055E0FFF71FFA00EBC00101EB4F
:101C7000001061684900B0FBF1F0B0FBF5F006011F
:101C8000FFF712FA00EBC00101EB00106168490098
:101C9000B0FBF1F7FFF708FA00EBC00101EB001011
:101CA00061684900B0FBF1F0B0FBF5F06FF018018E
:101CB000484307EB800108EBC100B0FBF5F000F0F2
:101CC000F80006EB4006FFF7EFF900EBC00101EB6F
:101CD000001061684900B0FBF1F7FFF7E5F900EB90
:101CE000C00101EB001061684900B0FBF1F0B0FBEE
:101CF000F5F06FF01801484307EB800108EBC100D5
:101D0000B0FBF5F000F00700216830448860BDE8C2
:101D1000F081FFF7C9F900EBC00101EB0010616829
:101D20008900B0FBF1F6FFF7BFF900EBC00101EB52
:101D3000001061688900B0FBF1F0B0FBF5F06FF0C6
:101D40001801484306EB800108EB0110B0FBF5F0E9
:101D500000F0F006FFF7A8F900EBC00101EB00105E
:101D600061688900B0FBF1F0B0FBF5F006EB0016FE
:101D7000FFF79AF900EBC00101EB001061688900E0
:101D8000B0FBF1F7FFF790F900EBC00101EB001099
:101D900061688900B0FBF1F0B0FBF5F06FF018015D
:101DA000484307EB800108EB0110B0FBF5F000F0B1
:101DB0000F00A9E7001401400010014090F839100D
:101DC000212901D0022070478168B1F5805F016A46
:101DD0000BD04A1C0262026809785160C18C491E0E
:101DE0000904090CC1840ED017E009880268C1F308
:101DF0000801516001690029016A02D0491C016291
:101E0000ECE7891CFBE70168CA6822F08002CA601F
:101E10000068C16841F04001C160002070472DE9B1
:101E2000F041984617460E460446069D1DE0681C84
:101E30001BD02DB1FFF700F8A0EB0800A84214D981
:101E40002068C16821F4D071C1602068416921F027
:101E500001014161202084F8390084F83A00002013
:101E600084F838000320BDE8F0812068006836EA75
:101E7000000004D00020B842D9D00020F3E70120B0
:101E8000F9E700000148FFF705BB0000B0000020A3
:101E90000148FFF7FFBA0000F0000020FEE7090745
:101EA000090E002804DB00F1E02080F800147047E0
:101EB00000F00F0000F1E02080F8141D704702E0F0
:101EC00008C8121F08C1002AFAD1704770470020C5
:101ED00001E001C1121F002AFBD170472DED088BD4
:101EE000FEF7B8FFFFF742FDFFF7A6FCFFF71CFD6A
:101EF000FFF7E2FCFFF7FCFCFFF76EFC314C9FEDB7
:101F000032AB9FED33BB42F210753348FEF71CFE37
:101F100032213148FEF7C6FD2F48FEF763FD8005EC
:101F200045D52D48FEF760FD80B200EE100ADFEDCA
:101F30002B0A2080B8EE400A20EE200ADFED280AA6
:101F400020EE200A84ED040A94ED018AB4EEC80A5A
:101F5000F1EE10FA30EE480A10EE100A08DDFEF736
:101F6000FCFA94ED020A41EC190B30EE480A07E046
:101F7000FEF7F3FA94ED030A41EC190B38EE400A30
:101F800010EE100AFEF7E9FA41EC100B51EC1A0BB7
:101F900053EC102BFEF772FA53EC192BFEF7FCF9F9
:101FA00053EC1B2BFEF7F5F9FEF7EAFA60610549E1
:101FB0000A23042214310B48FFF7AFFB2846FEF733
:101FC0004BFEA2E7000000200000000000000840D7
:101FD0000000000000001C40280000203333534064
:101FE00000008039700000200000000000000000A8
:101FF00001020304060708090000000001020304AF
:10200000202000080000002028000000BE1E00085C
:10201000482000082800002008410000CE1E0008CB
:10202000000000000000C03F85EB01409A99793F15
:10203000000000000000000001000000100000008F
:08204000000000000024F40080
:040000050800018965
:00000001FF
